:020000040800F2
:1000000000040020E1010008E3010008E30100080A
:10001000E3010008E3010008E3010008E301000830
:10002000E3010008E3010008E30100086D26000871
:10003000E3010008E3010008E3010008E301000810
:10004000E3010008E3010008E3010008E301000800
:10005000E3010008E3010008D53700080138000873
:100060002D3800085938000885380008E3010008D9
:10007000E3010008E3010008E3010008E3010008D0
:10008000E3010008E3010008E3010008E3010008C0
:10009000E3010008E3010008E3010008B1380008AB
:1000A000E3010008E3010008E3010008E3010008A0
:1000B000E3010008E3010008E3010008E301000890
:1000C000E3010008E3010008E3010008E301000880
:1000D000E3010008E3010008FD0F0008111000080B
:1000E00019390008E3010008E3010008E3010008F2
:1000F000E3010008E3010008E3010008E301000850
:10010000E3010008E3010008E5350008E301000809
:10011000E3010008E3010008E3010008E30100082F
:10012000E3010008E3010008E3010008E30100081F
:10013000E3010008E3010008E3010008E30100080F
:10014000E3010008E3010008E3010008592D00085D
:10015000E3010008E3010008E3010008E3010008EF
:10016000E3010008E3010008E3010008E3010008DF
:10017000E3010008E3010008E3010008E3010008CF
:10018000E3010008E301000825100008E30100086E
:10019000E3010008E3010008E3010008E3010008AF
:1001A000E3010008E3010008E3010008E30100089F
:1001B000E3010008E3010008E3010008E30100088F
:1001C000E3010008E3010008E3010008E30100087F
:1001D000E3010008E3010008E3010008E30100086F
:1001E00002E000F000F8FEE772B6394880F30888B4
:1001F000384880F3098838484EF60851CEF200019D
:10020000086040F20000CCF200004EF63471CEF2ED
:1002100000010860BFF34F8FBFF36F8F40F2000003
:10022000C0F2F0004EF68851CEF200010860BFF334
:100230004F8FBFF36F8F4FF00000E1EE100A4EF6C4
:100240003C71CEF200010860062080F31488BFF3F1
:100250006F8F02F049FA03F05BF94FF055301F49F8
:100260001B4A91423CBF41F8040BFAE71C49194A6A
:1002700091423CBF41F8040BFAE71A491A4A1B4B5A
:100280009A423EBF51F8040B42F8040BF8E70020F5
:100290001749184A91423CBF41F8040BFAE702F0B3
:1002A00027FA03F091F9144C144DAC4203DA54F8D8
:1002B000041B8847F9E700F03FF8114C114DAC42A0
:1002C00003DA54F8041B8847F9E702F00FBA00007C
:1002D000000400200024002000000008000000208E
:1002E00000040020E03D0008002400202824002015
:1002F0002824002090410020E0010008E0010008CF
:10030000E0010008E00100082DE9F04F2DED108A12
:10031000C1F80CD0C3689D46BDEC108ABDE8F08FD3
:10032000002383F311882846A047002001F058FEDF
:1003300001F008FE00DFFEE770B5204C0923002520
:1003400023706FF03F061F236570A570E57025715F
:100350006571A571E57125726672A372E57200F090
:10036000CBFC20B10F2325726672A372E57202F0F6
:100370004BF9044602F074F90546D8B9104B9C427B
:100380001AD001339C4218BF054641F2883404BF9D
:1003900001250024002002F03DF90DB100F0B6F86F
:1003A00000F02EFD00F0E6FB204600F00DF900F015
:1003B000ADF8F9E70024EDE70446EBE72824002038
:1003C000010007B008B500F053FBA0F1200358422C
:1003D000584108BD07B5054B02211B88ADF8043014
:1003E00001A800F0B1FB03B05DF804FB183A000867
:1003F000064991F8243033B100230822086A81F8B5
:10040000243000F0D9BB0120704700BF48240020F1
:100410002DE9F84F234C94F82430054688461746BA
:100420008BBB2E46DFF87C90002F38D094F824A0A8
:10043000BAF1000F05D12022FF214846266200F0C4
:10044000CDFCCAF10805BD4228BF3D465FFA85FBD9
:10045000AD0041462A4604EB8A0000F095FC94F872
:100460002430A7EB0B079B445FFA8BFBBBF1080F13
:100470002E44A844FFB284F824B0D5D1FFF7B8FFCA
:100480000028D1D108E0266A06EB8306B042C9D025
:10049000FFF7AEFF0028C4D10020BDE8F88F01208F
:1004A000BDE8F88F4824002010B5202383F311887D
:1004B0001248C3680BB101F019FE0023104A0F481F
:1004C0004FF47A7101F0D6FD002383F311880D4CAF
:1004D000236813B12368013B2360636813B1636829
:1004E000013B6360084B1B7833B9636823B9022072
:1004F00000F040FC3223636010BD00BF34240020B4
:10050000A9040008782900207024002010B5254B8C
:10051000254953F8042F013200D110BD8B42F8D188
:10052000224C234B22689A423AD9224B9B6803F112
:10053000006303F580439A4232D2002000F034FB7E
:100540001D4B0220187000F00BFC1C4B1A6C002293
:100550001A64196E1A66196E596C5A64596E5A6685
:100560005A6E5A6942F080025A615A6922F080023A
:100570005A615A691A6942F000521A611A6922F0E6
:1005800000521A611B6972B60D4A0E4B13601B684C
:100590002268202181F311889D4683F30888104743
:1005A00010BD00BFFC3F00081C40000804400008CC
:1005B000FF3F00082824002070240020003802405B
:1005C00008ED00E0004000082DE9F04FB54C97B071
:1005D00020228246FF210EA8A56800F0FFFBB24A48
:1005E0001378A046A3B9B1480121C360117020233C
:1005F00083F31188C3680BB101F078FD0023AC4A86
:10060000AA484FF47A7101F035FD002383F3118875
:10061000DFF8BCB2BAF1000F01D0CBF800A0A54FB3
:1006200000243C70CBF804402646012000F098FBE3
:10063000BAF1000F00F0E081DBF80030002B40F051
:10064000DB8117B0BDE8F08F0220FFF7BBFE00286A
:1006500040F0D081984B1B88ADF82430022109A8C6
:1006600000F072FAE1E74FF47A7000F001FA031E2D
:100670000193EFDB0220FFF7A5FE81460028E9D0B9
:10068000019B581E0428E5D8DFE800F0030C0F1288
:10069000150016A8052340F8343D042100F054FA53
:1006A0004C4650E004217F48F8E704218348F5E7F1
:1006B00004218348F2E71C24204600F077FA043432
:1006C0000990042109A800F03FFA2C2CF4D1E7E7A7
:1006D000002EBFD0002CBDD00220FFF773FE0646CF
:1006E00010B901242646B5E7012000F05DFA02208A
:1006F000387000F035FB0024E3B21846019300F097
:1007000063FA814648B1019B184600F06DFA013446
:100710000028F1D134466B4B9DE7012302203B704A
:1007200000F014FB4D46D8F808309D4206D228460A
:1007300000F03CFA0130EDD10435F4E700253D70BE
:10074000CBF80450344600F051FBFFF743FE4EE176
:10075000002E3FF47FAF002C3FF47CAF02203870B6
:1007600000F0FEFA322000F083F9041EB9DB14F029
:100770000306B6D1D8F808202B199342B1D8B4F5A6
:10078000807FAED8DFF84091A6420CDA4FF47A7041
:1007900000F06EF90390039B002BA2DB039B06F88D
:1007A00009300136F0E7C820FFF70CFE06460028A6
:1007B00097D01F2D11D8C5F12009A14528BFA1460A
:1007C0000EAB25F003004A463F49184400F0DCFA1E
:1007D0004A46FF213C4800F001FB4FEAA4095FFABA
:1007E00089F239492846FFF713FE0446002891D0C4
:1007F00005EB89050646A6E70220FFF7E3FD002882
:100800003FF428AFFFF7F4FD00283FF423AF4FF08B
:10081000000AD146D8F808309A453CD2BAF11F0FE9
:100820001CD80E9B013319D02AF0030316AA1344D7
:1008300053F8203C099325494B68A3B1002209A82D
:10084000135C83EA0903DBB2013251F82330042A36
:1008500083EA1929F4D10AF1040ADBE7504600F0D3
:10086000A5F90990E7E71A46082012F0010F4FEAB0
:1008700052021FBF82F06D4282F4380282F40342BA
:1008800082F020020138F0D141F823200133B3F582
:10089000807FE8D1D2E716A8042140F8489D00F0F7
:1008A00053F950E728240020742500203424002028
:1008B000A9040008702400201A3A00082C24002003
:1008C000302400201C3A00087424002078250020E1
:1008D0007829002016A8002340F8343D642100F058
:1008E000FFF800287FF4B6AE0220FFF76BFD00286A
:1008F0003FF4B0AE099800F089F916AB43F8440D07
:1009000004211846CBE716A8002340F8343D6421A3
:1009100000F0E6F800287FF49DAE0220FFF752FDBC
:1009200000283FF497AE099800F07EF916AB43F823
:10093000400DE5E70220FFF745FD00283FF48AAEB1
:1009400000F078F916AB43F83C0DD9E70220FFF729
:1009500039FD00283FF47EAE09A9142000F070F99B
:10096000814616A8042140F8389D00F0EDF849466C
:1009700009A894E74FF47A70FFF724FD00283FF4AC
:1009800069AEFFF735FD00283FF4C5AE0E9B01337D
:100990000CD008220EA90020FFF73AFD00283FF4F2
:1009A000BAAE2022FF210EA800F018FAFFF712FDC0
:1009B0002E4801F01BFB44E616A8002340F8343D06
:1009C000642100F08DF800287FF444AE0220FFF788
:1009D000F9FC00283FF43EAEFFF7FCFC41F2883002
:1009E00001F004FB099800F045FA00F0FFF94FF020
:1009F000000A1AE60646A6E6002000F039F8039041
:100A0000039B002BFFF614AE012000F09FF9039B1F
:100A1000213B122B3FF609AE01A252F823F000BF92
:100A20004906000867060008D10600082B060008E2
:100A30002B0600082B060008510700082B060008AB
:100A4000F9070008D508000807090008350900085B
:100A50002B0600084D0900082B0600087509000840
:100A6000470700082B060008B9090008A086010006
:100A70002DE9F34702AE00244FF47A7506F8014DD4
:100A8000144FDFF85880454397F900305A1C5FFA3D
:100A900084F901D0A34212D158F82400036801223E
:100AA000D3F820A031462B46D047012807D10A4B66
:100AB0009DF8070083F8009002B0BDE8F08701348C
:100AC000042CE1D14FF4FA7001F090FA4FF0FF30AE
:100AD000F2E700BF0024002098290020703A0008A7
:100AE0002DE9F0474FF47A75144FDFF85880064629
:100AF0004D43002497F900305A1C5FFA84F901D065
:100B0000A34210D158F8240003680422D3F820A08F
:100B100031462B46D047042805D1094B83F8009075
:100B20000020BDE8F0870134042CE3D14FF4FA70C3
:100B300001F05CFA4FF0FF30BDE8F08700240020A0
:100B400098290020703A000830B4074B1A78074BF8
:100B500053F822402368DD69054B0A46AC4601463E
:100B6000204630BC604700BF98290020703A00083A
:100B7000A086010070B501F081FC094C094E20707F
:100B8000002530682378834208D901F071FC33686E
:100B900005440133B5F5804F3360F2D370BD00BF1B
:100BA000992900208029002001F01ABD00F1006081
:100BB00000F580400068704700F10060920000F589
:100BC000804001F0A5BC0000054B1A68054B1B785E
:100BD0009B1A834202D9104401F04ABC002070479E
:100BE000802900209929002038B5074D044628683F
:100BF000204401F045FC28B928682044BDE838406D
:100C000001F056BC38BD00BF8029002010F003035E
:100C100008D1B0F5007F05D800F10050A0F50840DC
:100C20000068704700207047014BC058704700BFF4
:100C3000107AFF1F014B1868704700BF002004E0C6
:100C400070B52A4B1C68C4F30B03240C63B140F24B
:100C50001342934231D040F2194293422FD040F2D6
:100C6000214293422DD10323214A0C2505FB032366
:100C70005D6893F9082042F201039C4224D0B4F548
:100C8000805F23D041F201039C4221D041F2030353
:100C90009C421FD041F207039C4208BF3122441EF0
:100CA0000C44013D0B46A3421ED215F9016F581C9E
:100CB00096B1034600F8016CF5E70123D4E702235F
:100CC000D2E73F220B4DD6E73322E3E74122E1E7AB
:100CD0005A22E4E75922E2E72C2584421D7001D90B
:100CE000981C5A70401A70BD1846FBE7002004E0BB
:100CF000403A0008203A0008124B5A8842F201019B
:100D00008A4293B214D0B3F5805F13D041F201024E
:100D1000934211D041F2030293420FD041F20702F5
:100D200093420DD10423084A02EB8303D87870471D
:100D30000023F8E70123F6E70223F4E70323F2E7B1
:100D400000207047002004E02C3A0008022802BF6F
:100D5000024B4FF480529A61704700BF001002406E
:100D6000022802BF024B4FF080529A61704700BFC9
:100D700000100240022801BF024A536983F48053E5
:100D8000536170470010024010B50023934203D016
:100D9000CC5CC4540133F9E710BD000030B5441EEB
:100DA00014F9010F0B4660B193F90050854201F12F
:100DB000010106D11AB993F90020801A30BD013A19
:100DC000EEE7002AF7D1104630BD00000246034688
:100DD000981A13F9011B0029FAD1704702440346FF
:100DE000934202D003F8011BFAE77047024B1A78CE
:100DF000024B1A70704700BF982900200024002081
:100E0000F8B5164C1648174D174E154F00F036FC26
:100E10002146134800F05EFC236814485A6D936B1A
:100E200023F40023936301F0E1F82068104900F0F7
:100E30005DFD23685A6D936B43F4002393634FF475
:100E4000E1332B60002456F82400B84202D0294632
:100E500000F072FB0134042CF5D1F8BD583B0008BA
:100E60001437002084290020703A000840420F0007
:100E7000B03B000838B50B4B1A780B4B53F82240A7
:100E80000A4B9C4205460CD0094B002118461422FF
:100E9000FFF7A4FF056001462046BDE8384000F09A
:100EA0004BBB38BD98290020703A00081437002049
:100EB00084290020026843681143016003B1184788
:100EC00070470000024AD36843F0C003D360704704
:100ED00000440040024AD36843F0C003D360704727
:100EE00000480040024AD36843F0C003D360704713
:100EF000007800402DE9F041D0F85C64F768336871
:100F0000DA0505469CB20DD5202383F311884FF4F2
:100F100000710430FFF7CEFF6FF48073336000235D
:100F200083F31188202383F3118805F1040814F05A
:100F30002F0333D183F31188380615D5210613D535
:100F4000202383F3118805F1380000F053FA0028BC
:100F500046DA0821281DFFF7ADFF4FF67F733B40AF
:100F6000F360002383F311887A060ED563060CD54F
:100F7000202383F31188EA6C2B6D9A4202D12B6CEB
:100F8000002B2FD1002383F31188D5F86424D36874
:100F9000002B31D01069BDE8F0411847230713D06A
:100FA00014F0080F0CBF00218021E00748BF41F07A
:100FB0002001A20748BF41F04001630748BF41F448
:100FC00080714046FFF776FFA406736805D595F853
:100FD00060142846194000F0BDFA3468A4B2A6E7B0
:100FE0007060BEE727F040073F041021281D3F0C2A
:100FF000FFF760FFF760C5E7BDE8F08108B503487B
:10100000FFF778FFBDE8084001F040BB9C290020B5
:1010100008B50348FFF76EFFBDE8084001F036BB96
:10102000042E002008B50348FFF764FFBDE8084020
:1010300001F02CBB6C32002010B50E4C0E4A20463D
:10104000002100F057FA0D4BC4F85C340C4C0D4AEB
:101050002046002100F04EFA0B4BC4F85C340B4CD8
:101060000B4A0021204600F045FA0A4BC4F85C34D4
:1010700010BD00BF9C290020C50E000800440040A0
:10108000042E0020D50E0008004800406C320020DD
:10109000E50E00080078004038B5394D037C002982
:1010A00018BF0D46012B0446C0F8645410D1354BCF
:1010B000984242D1344B1A6C42F400321A641A6ED0
:1010C00042F400321A661B6E0B21262000F06AF8EB
:1010D0002E4BD4F85C249A422B6802D02C498A42C9
:1010E0004BD12C4901EB5301B1FBF3F3A988080460
:1010F00042BF23F0070003F0070343EA4003936075
:10110000EB8843F040039BB213612B8943F001034A
:101110009BB2536141F4045343F02C03D36001F4B8
:10112000A05100231360B1F5806F136853680CBFA2
:101130007F23FF2384F8603438BD174B98420CD1CD
:10114000114B1A6C42F480221A641A6E42F4802207
:101150001A661B6E0B212720B8E7104B9842B7D1B7
:10116000094B1A6C42F080421A641A6E42F08042B7
:101170001A661B6E0B215220A8E70949B2E700BF8F
:10118000A03A00089C2900200038024000100140CD
:101190000014014000BD0105042E00206C32002027
:1011A00080DE800200F1604300F01F02400903F579
:1011B000614309018000C9B200F1604083F8001367
:1011C00000F5614001239340C0F88031036070470F
:1011D000F8B5154682680669AA420B46816938BF90
:1011E0008568761AB542044607D218462A46FFF7A4
:1011F000CBFDA3692B44A3610DE011D932461846FB
:10120000FFF7C2FDAF1B3A46E1683044FFF7BCFD73
:10121000E2683A44A261A3685B1BA3602846F8BD5C
:1012200018462A46FFF7B0FDE368E4E783682DE936
:10123000F041044693421546266938BF85684069E7
:10124000361AB5420F4606D22A46FFF79DFD63695E
:101250002B4463610DE012D93246A5EB0608FFF777
:1012600093FD4246B919E068FFF78EFDE2684244FB
:101270006261A3685B1BA3602846BDE8F0812A4633
:10128000FFF782FDE368E4E710B50A440024C36178
:10129000029B006040608460C160816141610261C5
:1012A000036210BD08B582694369934201D1826827
:1012B00082B98268013282605A1C426119704269A7
:1012C00003699A4201D3C3684361002100F0AAFE7A
:1012D000002008BD4FF0FF3008BD000070B520238E
:1012E00004460E4683F31188A568A5B1A368A269D8
:1012F000013BA360531CA36115782269934224BF6C
:10130000E368A361E3690BB120469847002383F3A8
:101310001188284670BD3146204600F073FE002833
:10132000E2DA85F3118870BD2DE9F74F05460F46C7
:1013300090469A46D0F81C90202686F311884FF0EC
:10134000000B144664B1224639462846FFF740FF99
:10135000034668B95146284600F054FE0028F1D0F3
:10136000002383F31188A8EB040003B0BDE8F08FDD
:10137000B9F1000F03D001902846C847019B8BF3B9
:101380001188E41A1F4486F31188DBE7C16081618C
:101390004161C3611144009B006040608260016153
:1013A00003627047F8B504460E461746202383F3C0
:1013B0001188A568A5B1A368013BA36063695A1CA5
:1013C00062611E70236962699A4224BFE3686361A7
:1013D000E3690BB120469847002080F31188F8BDDF
:1013E0003946204600F00EFE0028E2DA85F3118827
:1013F000F8BD0000836942699A4210B501D1826844
:101400007AB98268013282605A1C82611C78036951
:101410009A4201D3C3688361002100F003FE204695
:1014200010BD4FF0FF3010BD2DE9F74F05460F46B8
:1014300090469A46D0F81C90202686F311884FF0EB
:10144000000B144664B1224639462846FFF7EEFEEB
:10145000034668B95146284600F0D4FD0028F1D073
:10146000002383F31188A8EB040003B0BDE8F08FDC
:10147000B9F1000F03D001902846C847019B8BF3B8
:101480001188E41A1F4486F31188DBE70268436879
:101490001143016003B11847704700001430FFF793
:1014A00043BF00004FF0FF331430FFF73DBF000093
:1014B0003830FFF7B9BF00004FF0FF333830FFF787
:1014C000B3BF00001430FFF709BF00004FF0FF3139
:1014D0001430FFF703BF00003830FFF763BF000090
:1014E0004FF0FF323830FFF75DBF0000002070473B
:1014F000FFF7A2BD37B50F4B036000234360836045
:10150000C360012304460374154600900B464FF454
:10151000007200F15C011430FFF7B6FE00942B4618
:101520004FF4007204F5177104F13800FFF72EFF35
:1015300003B030BDB43A000810B52023044683F34D
:101540001188FFF7A9FD02232374002383F3118878
:1015500010BD000038B5C36904460D461BB904210F
:101560000844FFF793FF294604F11400FFF79AFEA1
:10157000002806DA201D4FF48061BDE83840FFF7EF
:1015800085BF38BD026843681143016003B1184745
:101590007047000013B5446BD4F894341A6811787E
:1015A000042915D1217C022912D11979128901232C
:1015B0008B4013420CD101A904F14C0001F01CFE38
:1015C000D4F89444019B21790246206800F0DAF9AE
:1015D00002B010BD143001F09FBD00004FF0FF338A
:1015E000143001F099BD00004C3001F071BE0000D4
:1015F0004FF0FF334C3001F06BBE0000143001F0AF
:101600006DBD00004FF0FF31143001F067BD0000E8
:101610004C3001F03DBE00004FF0FF324C3001F085
:1016200037BE0000D0F8942438B51368197804291F
:10163000054601D0012038BD017C0229FAD112797A
:101640005C89012090400440F4D105F1140001F0C0
:10165000FFFC02460028EDD0D5F894544FF4807377
:101660002868697900F07CF9204638BD406BFFF7A7
:10167000D9BF000000207047704700007FB5124BB3
:101680000360002343608360C360012502260F4B83
:10169000057404460290019300F1840229460096E5
:1016A0004FF48073143001F0AFFC094B01930294A6
:1016B00000964FF4807304F52372294604F14C0020
:1016C00001F076FD04B070BDDC3A00086D1600082C
:1016D000951500080B68202282F311880A7903EB24
:1016E000820290614A79093243F822008A7912B164
:1016F00003EB8203986102230374C0F8941400235F
:1017000083F311887047000038B5037F044613B196
:1017100090F85430ABB9201D01250221FFF732FFAC
:1017200004F1140025776FF0010100F087FC84F8C4
:10173000545004F14C006FF00101BDE8384000F056
:101740007DBC38BD10B5012104460430FFF71AFFF7
:101750000023237784F8543010BD000038B50446C8
:101760000025143001F068FC04F14C00257701F0ED
:1017700037FD201D84F854500121FFF703FF204658
:10178000BDE83840FFF74EBF90F8443003F06003E7
:10179000202B19D190F84520212A0AD0222A4FF077
:1017A00000030ED0202A0FD1084A82630722C263A9
:1017B00004E0064B83630723C36300230364012013
:1017C00070478363C363F9E700207047012400205A
:1017D000D0F8943437B51A681178042904461AD120
:1017E000017C022917D11979128901238B401342F8
:1017F00011D100F14C05284601F0B2FD58B101A904
:10180000284601F0F9FCD4F89444019B2179024662
:10181000206800F0B7F803B030BD000000EB810392
:10182000F7B59C6905460E46F4B1202383F3118871
:1018300005EB8607201D0821FFF7A4FEFB685B6906
:101840001B684C3413B1204601F0E4FC01A920468A
:1018500001F0D2FC024648B1019B3146284600F017
:1018600091F8002383F3118803B0F0BDFB685A6937
:101870001268002AF5D01B8A013B1340F1D105F113
:101880004402EAE7093138B550F82140DCB12023A1
:1018900083F31188D4F894241368527903EB8203FC
:1018A000DB689B695D6845B104216018FFF76AFE3B
:1018B000294604F1140001F0D5FB2046FFF7B2FEE3
:1018C000002383F3118838BD7047000000F096BFF5
:1018D0000123037000234360C36183620362C36218
:1018E00043620363038143817047000038B50446B7
:1018F000202383F3118800254160C560056145619F
:10190000856100F08BFF0223237085F3118838BDB9
:1019100070B500EB810305465069DA600E46144647
:1019200018B110220021FFF759FAA06918B110224E
:101930000021FFF753FA31462846BDE8704001F018
:1019400037B80000028902F001020281428902F0E8
:1019500001024281002202614261826101F0BCB851
:10196000F0B400EB81044789E4680125A4698D4047
:101970003D43458123600023A2606360F0BC01F019
:10198000D7B80000F0B400EB81040789E4680125B2
:1019900064698D403D43058123600023A26063603C
:1019A000F0BC01F051B9000070B5022300250446D7
:1019B0000370A0F84C5080F84E5080F84F500581CD
:1019C0004581C56005614561856180F8345000F04E
:1019D0008BFF63681B6823B129462046BDE8704031
:1019E000184770BD436802781B6880F850200522B4
:1019F00002700BB10421184770470000436890F84B
:101A000050201B6802700BB1052118477047000079
:101A100090F8343070B5044613B1002380F83430A8
:101A200004F14402204601F079F863689B6863BBC7
:101A300094F8445015F0600615D194F8453005F03F
:101A40007F0545EA032540F202339D4200F00E81F6
:101A50005BD8022D00F0DC803FD8002D00F087809D
:101A6000012D00F0CF800021204601F0AFFA0021C7
:101A7000204601F0A1FA63681B6813B106212046D5
:101A80009847062384F8343070BD204698470028D4
:101A9000CED094F84B2094F84A3043EA0223E26B0C
:101AA000934238BFE36394F94430E56B002B4FF069
:101AB000200380F2FD80002D00F0EC80092284F8E4
:101AC000342083F311880021E36BA26B2046FFF7DB
:101AD00059FF002383F3118870BDB5F5817F00F0B5
:101AE000B180B5F5407F49D0B5F5807FBBD194F882
:101AF0004630012BB7D1B4F84C3023F00203A4F8E0
:101B00004C30A663E6632664C3E740F201639D425E
:101B10001ED8B5F5C06F3BD2B5F5A06FA3D1B4F810
:101B20004430B3F5A06F0ED194F8463084F84E30AF
:101B3000204600F031FF63681B6813B10121204685
:101B40009847032323700023A363E3632364A0E780
:101B5000B5F5106F32D040F602439D4252D0B5F534
:101B6000006F80D104F14F03A363012324E004F14B
:101B70004C03A3630223E36325648AE794F84630A9
:101B8000012B7FF470AFB4F84C3043F00203B6E79A
:101B900094F84920616894F848304D6894F84710EB
:101BA00043EA0223204694F84620A84700283FF441
:101BB0005AAF4368A3630368E363A4E72378042B65
:101BC00010D1202383F311882046FFF7BBFE86F354
:101BD0001188636884F84F601B68032121700BB182
:101BE0002046984794F84630002BACD084F84F300C
:101BF0000423237063681B68002BA4D002212046B5
:101C00009847A0E7374BA3630223E36300239DE7D4
:101C100094F8481011F0800F204601F00F010ED00B
:101C200000F06EFF012806D002287FF41CAF2E4B77
:101C3000A363E06367E72D4BA363E56363E700F00D
:101C400051FFEFE794F84630002B7FF40CAF94F887
:101C5000483013F00F013FF476AF1A06204602D544
:101C600001F0C8F96FE701F0BBF96CE794F8463072
:101C7000002B7FF4F8AE94F8483013F00F013FF4D6
:101C800062AF1B06204602D501F0A0F95BE701F028
:101C900093F958E7142284F8342083F311882B46F3
:101CA0002A4629462046FFF75BFE85F3118870BD62
:101CB0005DB1152284F8342083F311880021E36B91
:101CC000A26B2046FFF74CFE03E70B2284F834207A
:101CD00083F311882B462A4629462046FFF752FEF9
:101CE000E3E700BF0C3B0008043B0008083B00088A
:101CF00038B590F834300446152B29D8DFE803F0C6
:101D00003E28282828283E28280B29392828282832
:101D1000282828283E3E90F84B1090F84A20C36BA4
:101D200042EA01229A4214D9C268128AB3FBF2F540
:101D300002FB15356DB9202383F311882B462A4603
:101D40002946FFF71FFE85F311880A2384F83430F3
:101D500038BD142384F83430202383F31188002302
:101D60001A4619462046FFF7FBFD002383F311882E
:101D700038BD036C03B198470023E7E7002101F069
:101D800025F90021204601F017F963681B6813B19B
:101D90000621204698470623D8E7000090F8342013
:101DA000152A38B5044622D80123934040F64162F3
:101DB00013421DD113F480150FD19B0217D50B23AD
:101DC00080F83430202383F311882B462A46294695
:101DD000FFF7D8FD85F3118838BDC3689B695B6840
:101DE0002BB9036C03B19847002384F8343038BD15
:101DF000002101F0EBF80021204601F0DDF86368D6
:101E00001B6813B10621204698470623EDE7000022
:101E1000024B00221B605B609A607047D436002042
:101E2000002303748268054B1B6899689142FBD2BA
:101E30005A6803604260106058607047D4360020D2
:101E400008B5202383F31188037C032B05D0042BD2
:101E50000DD02BB983F3118808BD436900221A60A5
:101E60004FF0FF334361FFF7DBFF0023F2E790E819
:101E70000C001A6002685360F2E70000002303744C
:101E80008268054B1B6899689142FBD85A680360C9
:101E90004260106058607047D4360020054B1969C5
:101EA0000874186802681A6053601861012303748B
:101EB000FEF72ABAD436002030B54B1C87B0054651
:101EC0000A4C10D023690A4A01A800F0D3F828462A
:101ED000FFF7E4FF049B13B101A800F007F92369A1
:101EE000586907B030BDFFF7D9FFF8E7D4360020B6
:101EF000411E000838B50C4D41612B6981689A6814
:101F00009142044603D8BDE83840FFF789BF184620
:101F1000FFF786FF01232C61014623742046BDE8AC
:101F20003840FEF7F1B900BFD4360020044B1A68E0
:101F30001B6990689B68984294BF002001207047FD
:101F4000D436002010B5084C236820691A68226036
:101F50005460012223611A74FFF790FF0146206943
:101F6000BDE81040FEF7D0B9D436002082600222CE
:101F700002740022427470478368A3F17C0243F824
:101F80000C2C026943F83C2C426943F8382C074A70
:101F900043F81C2CC26843F8102C022203F8082CCA
:101FA000002203F8072CA3F1180070472103000852
:101FB00010B5202383F31188FFF7DEFF00210446CC
:101FC000FFF798FF002383F31188204610BD00001F
:101FD000024B1B6958610F20FFF760BFD436002009
:101FE000202383F31188FFF7F3BF000008B50146F3
:101FF000202383F311880820FFF75EFF002383F37B
:10200000118808BD49B1064B42681B6918605A60C7
:10201000136043600420FFF74FBF4FF0FF3070475D
:10202000D43600200368984206D01A6802605060D7
:1020300059611846FFF7F4BE7047000038B50446F2
:102040000D462068844200D138BD036823605C607F
:102050004561FFF7E5FEF4E7054B03F114025A6111
:102060009A614FF0FF32DA6100221A62704700BFB6
:10207000D4360020F8B503611A4BC2605C6A1A4B73
:102080001A46022952F8145F38BF022195420646CB
:102090001F460AD1586198611C62056045608160E5
:1020A0000819BDE8F84001F07DB9186AAB68241A38
:1020B0000C1902D3E41A2D6804E09C4202D2204499
:1020C00001F080F9AB689C42F4D86B6873603560AE
:1020D0001E606E60B460A9684FF0FF33091BA960F1
:1020E000FB61F8BD000C0040D436002010B41A4C3F
:1020F000234653F8141F814210D0416802680A60D9
:10210000026851609A424FF00001C16003D09368A9
:1021100081680B4493605DF8044B70470A68626104
:1021200000209A425360C86003D15DF8044B01F06F
:1021300043B99368886803449360084A206A526AE6
:10214000121A9342E7D9991A012998BF931C18448F
:102150005DF8044B01F036B9D4360020000C004085
:1021600000207047FEE70000704700004FF0FF308E
:1021700070470000022906D0032906D0012906482D
:1021800018BF0020704705487047032A9ABF0448CB
:1021900000EBC200002070470C3C0008C03B000868
:1021A0000824002070B5044608460D46FEF70EFED2
:1021B000C6B22046013403780BB9184670BD3246CA
:1021C0002946FEF7EBFD0028F3D1012070BD000089
:1021D0002DE9F04F80469BB008460C461646FEF7A8
:1021E000F5FD3C49C5B22046FFF7DCFF08B10735D5
:1021F000EDB239492046FFF7D5FF08B11035EDB2F1
:10220000632D01AF0CD8DFF8DC90DFF8DCB03D4681
:1022100094F800A0BAF1000F1CD185F800A003E0EB
:102220002146384601F0F0FB3846FEF7CFFDC0B23C
:10223000431C5B0088E8480033700323737000235D
:1022400002361946DAB2904206F102063BD81BB0BC
:10225000BDE8F08FBAF1250F30D107221D49204685
:10226000FEF79CFD70B91D4B2A4603F10C0153F893
:10227000040B42F8040B8B42F9D11B8813800734FE
:102280000E35C5E7082214492046FEF787FDA8B998
:102290001349AB1C11F8012F100902F00F0210F8BE
:1022A000090012F8092003F8020C594503F8012C23
:1022B00003F10203EED118350834A9E785F800A030
:1022C00001340135A4E7FA5C06F8022C06F8011C7B
:1022D0000133B7E7603B0008683B0008713B00082A
:1022E0000F7AFF1F803B00081B7AFF1F08B52023D1
:1022F00083F311880348FFF76BFA002383F31188F7
:1023000008BD00BF1437002010B50446052916D8B3
:10231000DFE801F016150316161D202383F311883C
:102320000E4A0121FFF7F4FA20460D4A0221FFF779
:10233000EFFA0C48FFF712FA002383F3118810BD5F
:10234000202383F311880748FFF7DEF9F4E7202301
:1023500083F311880348FFF7F5F9EDE7103B000818
:10236000343B00081437002038B50C4D0C4C0D4997
:102370002A4604F10800FFF72BFF05F1CA0204F119
:1023800010000949FFF724FF05F5CA7204F118008F
:102390000649BDE83840FFF71BBF00BFDC3B00200B
:1023A00008240020943B0008A13B0008683B00087B
:1023B000BFF34F8F024AD368DB03FCD4704700BFE2
:1023C000003C024008B5094B1B7873B9FFF7F0FFDA
:1023D000074B1A69002ABFBF064A5A6002F18832C9
:1023E0005A601A6822F480621A6008BD3A3E0020E2
:1023F000003C02402301674508B50B4B1B7893B99D
:10240000FFF7D6FF094B1A6942F000421A611A68B9
:1024100042F480521A601A6822F480521A601A68D4
:1024200042F480621A6008BD3A3E0020003C02403F
:10243000172870B513D80B4A0B4C137863B90B4EA1
:102440004FF0006144F8231056F823500133182B45
:102450002944F7D10123137054F8200070BD0020E7
:1024600070BD00BF9C3E00203C3E00202C3C00087C
:10247000014B53F8200070472C3C0008182070478F
:10248000172810B5044601D9002010BDFFF7D0FF72
:10249000064B53F824301844C21A0BB9012010BD62
:1024A00012680132F0D1043BF6E700BF2C3C000873
:1024B000172810B5044626D8FFF77AFFFFF782FFEA
:1024C0001249F323CB60FFF773FF0C23B0FBF3F249
:1024D00003FB1200D30143EAC003DBB243F40073F1
:1024E00043F002030B610B6943F480330B61FFF788
:1024F0005FFF2046FFF79CFFFFF77EFF2046BDE809
:102500001040FFF7BDBF002010BD00BF003C0240DF
:102510002DE9F84312F00103154643D10244B2F10C
:10252000026F3FD22C4B1B6813F001033AD02B4CA7
:10253000FFF748FFF323E360FFF73AFF40F201277C
:10254000032D16D8254C0F46401A40F20118EB1BFC
:102550000B44012B00EB0706236926D823F0010367
:102560002361FFF749FF0120BDE8F883043D0430F3
:10257000E6E78307E6D1236923F4407323612369E7
:102580003B43236151F8046B0660BFF34F8FFFF7A5
:102590000FFF03689E42E9D0236923F00103236102
:1025A000FFF72AFF0020BDE8F88323F4407323617E
:1025B000236943EA08032361B94637F8023B3380B5
:1025C000BFF34F8FFFF7F4FE3688B9F80030B6B28C
:1025D000B342BCD0E0E700BF00380240003C0240FC
:1025E000084908B50B7828B153B9FFF7EBFE012372
:1025F0000B7008BD23B1BDE808400870FFF7FCBEB2
:1026000008BD00BF3A3E0020014B186D704700BF67
:1026100000280040094B1A6F120407D41A6F42F4C5
:1026200000721A671A6F42F400421A67044A13686C
:1026300043F480731360034B186570470038024001
:102640000070004000280040034B1B689B0042BF05
:10265000024B01221A707047743802409D3E0020E0
:10266000014B1878704700BF9D3E0020064A536812
:1026700023F001035360EFF30983683383F3098880
:10268000002383F31188704730EF00E010B520235A
:1026900083F31188104B5B6813F4006318D0F1EEDC
:1026A000103AEFF309844FF0807344F84C3C0B4B25
:1026B000DB6844F8083CA4F1680383F30988FFF75A
:1026C00035FC18B1064B44F8503C10BD054BFAE7F9
:1026D00083F3118810BD00BF00ED00E030EF00E093
:1026E000310300083403000870470000FEE70000D3
:1026F000084A094B09498B4204D3094A00219342F5
:1027000005D3704752F8040F43F8040BF3E743F87E
:10271000041BF4E7043E0008904100209041002093
:1027200090410020836D30B500229D68446D1146B4
:102730004FF0FF3004EB421301329542C3F8001909
:10274000C3F81019C3F80809C3F8001BC3F8101B1D
:10275000C3F8080BEED24FF00113C4F81C3830BD9B
:10276000890141F02001016103699B06FCD412201C
:1027700000F0B4BE204B03EB80022DE9F047D2F805
:102780000CE05D6DDEF81420461CD2F800C005EBAD
:10279000063605EB4018516861450BD3D5F834284F
:1027A000012303FA00F022EA0000C5F834081846B5
:1027B000BDE8F087BEF81040ACEB0103A34228BF90
:1027C0002346D8F81849A4B2B3EB840F10D8946804
:1027D0001F46A4F1040959F804AFC6F800A0042F5D
:1027E00001D9043FF7E71C440B4494605360D2E7DF
:1027F0000020BDE8F08700BFA03E002010B5054CCA
:102800002046FFF765F84FF0A0436365024BA365D0
:1028100010BD00BFA03E0020B03C00080378012B93
:1028200070B5054650D12A4B446D98421BD1294BB7
:102830005A6B42F080025A635A6D42F080025A6528
:102840005A6D5A6942F080025A615A6922F0800238
:102850005A610E2143205B69FEF7A4FC1E4BE36026
:102860001E4BC4F800380023C4F8003EC023236088
:102870006E6D4FF45023A3633369002BFCDA012300
:1028800033610C2000F02AFE3369DB07FCD41220F0
:1028900000F024FE3369002BFCDA0026A6602846EF
:1028A000FFF740FF6B68C4F81068DB68C4F8146871
:1028B000C4F81C684BB90A4BA3614FF0FF33636146
:1028C000A36843F00103A36070BD064BF4E700BFAB
:1028D000A03E0020003802404014004003002002C7
:1028E000003C30C0083C30C0F8B5446D05460021BE
:1028F0002046FFF735FFA96D00234FF001128F68C6
:10290000C4F834384FF00066C4F81C284FF0FF308C
:1029100004EB431201339F42C2F80069C2F8006B16
:10292000C2F80809C2F8080BF2D20B686A6DEB65B1
:10293000636210231361166916F01006FBD1122092
:1029400000F0CCFDD4F8003823F4FE63C4F800385E
:10295000A36943F4402343F01003A3610923C4F89F
:102960001038C4F814380A4BEB604FF0C043C4F879
:10297000103B084BC4F8003BC4F81069C4F8003998
:10298000EB6D03F1100243F48013EA65A362F8BD16
:102990008C3C000840800010426D90F84E10D2F838
:1029A000003823F4FE6343EA0113C2F8003870478D
:1029B0002DE9F0410EB200EB86080D46D8F80C1058
:1029C0000F6807F00303022B50D0032B50D03D4A71
:1029D0003D4F012B18BF1746446D4FEA451E04EBCF
:1029E0000E030022C3F8102B8A6905F1100C002A8F
:1029F00040D04A8A05F158035B013A43E250012373
:102A0000D4F81C2803FA0CF31343A6444A69C4F80B
:102A10001C380023CEF8103905F13F03002A39D0C5
:102A20000A8A898B9208012988BF4A43C16D04EB49
:102A30008303561841EA0242C66529465A60204679
:102A4000FFF78EFED8F80C301B8A43EA85531F43EC
:102A500005F148035B01E7500123D4F81C2803FA71
:102A600005F51543C4F81C58BDE8F081174FB3E7CE
:102A7000174FB1E704EB4613D3F8002B22F40042C2
:102A8000C3F8002BD4F81C28012303FA0CF322EA24
:102A90000303BAE704EB83030E4A5A6004EB4616BD
:102AA00029462046FFF75CFED6F8003923F40043A0
:102AB000C6F80039D4F81C38012202FA05F523EAD9
:102AC0000505CFE70080001000800410008008108A
:102AD00000800C1000040002826D1268C265FFF7CE
:102AE00021BE00005831436D49015B5813F400408A
:102AF00004D013F4001F14BF01200220704700000F
:102B00004831436D49015B5813F4004004D013F47D
:102B1000001F14BF012002207047000000EB81015C
:102B2000CB68196A0B6813604B68536070470000EC
:102B300000EB810330B5DD68AA691368D36019B969
:102B4000402B84BF402313606B8A1468426D1C4481
:102B5000013CB4FBF3F46343033323F0030302EBC0
:102B6000411043EAC44343F0C043C0F8103B2B6814
:102B700003F00303012B09B20ED1D2F8083802EB9F
:102B8000411013F4807FD0F8003B14BF43F0805312
:102B900043F00053C0F8003B02EB4112D2F8003B77
:102BA00043F00443C2F8003B30BD00002DE9F04182
:102BB000244D6E6D06EB40130446D3F8087BC3F832
:102BC000087B38070AD5D6F81438190706D505EB5F
:102BD00084032146DB6828465B689847FA072FD5AF
:102BE000D6F81438DB072BD505EB8403D968CCB9AC
:102BF0008B69488A5E68B6FBF0F200FB12628AB904
:102C00001868DA6890420DD2121A83E81400202363
:102C100083F311880B482146FFF78AFF84F311885C
:102C2000BDE8F081012303FA04F26B8923EA020371
:102C30006B81CB6823B121460248BDE8F0411847BB
:102C4000BDE8F081A03E002000EB810370B5DD6897
:102C5000436D6C692668E6604A0156BB1A444FF41E
:102C60000020C2F810092A6802F00302012A0AB201
:102C70000ED1D3F8080803EB421410F4807FD4F887
:102C8000000914BF40F0805040F00050C4F8000923
:102C900003EB4212D2F8000940F00440C2F80009E8
:102CA000D3F83408012202FA01F10143C3F83418C1
:102CB00070BD19B9402E84BF4020206020682E8A44
:102CC000841940F00050013C1A44B4FBF6F440EA89
:102CD000C440C6E7F8B504461E48456D05EB4413ED
:102CE000D3F80869C3F80869F10717D5D5F8103883
:102CF000DA0713D500EB8403D9684B691F68DA68DB
:102D0000974218D2D21B00271A605F60202383F3FA
:102D100011882146FFF798FF87F31188330617D5EE
:102D2000D5F834280123A340134211D02046BDE832
:102D3000F840FFF71FBD012303FA04F2038923EAD9
:102D4000020303818B68002BE8D021469847E5E712
:102D5000F8BD00BFA03E002096482DE9F84F456D14
:102D60006E69AB691E4016F4805F6E61044605D043
:102D7000FEF71AFEBDE8F84FFFF788BC002E12DA06
:102D8000D5F8003E8B489B071EBFD5F8003E23F0C8
:102D90000303C5F8003ED5F8043823F00103C5F855
:102DA0000438FEF72BFE370502D58248FEF71AFEDF
:102DB000B0040CD5D5F8083813F0060FEB6823F4EF
:102DC00070530CBF43F4105343F4A053EB6031072E
:102DD00004D56368DB680BB176489847F2025AD491
:102DE000B3020CD5D4F85480DFF8C8A100274FF007
:102DF0000109A36D9B68F9B28B4280F08780F706CA
:102E000019D5616D0A6AC2F30A1702F00F0302F4C2
:102E1000F012B2F5802F00F0A180B2F5402F0AD158
:102E200004EB830301F58051DB68186A00231A461E
:102E30009F4240F087803003D5F8184813D5E1034E
:102E400002D50020FFF7B2FEA20302D50120FFF752
:102E5000ADFE630302D50220FFF7A8FE270302D5CB
:102E60000320FFF7A3FE750384D5E00702D50020F9
:102E7000FFF730FFA10702D50120FFF72BFF620704
:102E800002D50220FFF726FF23077FF573AF03204B
:102E9000FFF720FF6EE7D4F85480DFF818A1002771
:102EA0004FF00109A36D9B685FFA87FB5B4597D3E1
:102EB00008EB4B13D3F8002902F44022B2F5802F1F
:102EC00022D1D3F80029002A1EDAD3F8002942F0D3
:102ED0009042C3F80029D3F80029002AFBDB5946A9
:102EE000606DFFF73DFC228909FA0BF322EA030328
:102EF000238104EB8B03DB689B6813B15946504672
:102F000098475846FFF736FC0137CBE708EB4112EC
:102F1000D2F8003B03F44023B3F5802F10D1D2F850
:102F2000003B002B0CDA628909FA01F322EA030361
:102F3000638104EB8103DB68DB680BB15046984783
:102F4000013756E79C0708BF0A68072B98BF027035
:102F500003F101039CBF120A013069E7023304EB5D
:102F6000830201F58051526890690268D0F808C068
:102F70004068A2EB000E0022104697420AD104EBF3
:102F8000830463689B699A683A449A605A68174454
:102F90005F6050E712F0030F08BF0868964588BFCE
:102FA0008CF8000002F1010284BF000A0CF1010C50
:102FB000E3E700BFA03E0020436D03EB4111D1F8D1
:102FC000003B43F40013C1F8003B7047436D03EB33
:102FD0004111D1F8003943F40013C1F800397047AA
:102FE000436D03EB4111D1F8003B23F40013C1F80A
:102FF000003B7047436D03EB4111D1F8003923F4D6
:103000000013C1F80039704730B5039C01720433D6
:1030100004FB0325C361049B03630021059B00603F
:103020004060C16042610261856104624262816206
:10303000C162436330BD00000022416A4161016109
:10304000C2608262C2626FF00101FEF7F7BF00004A
:1030500003694269934203D1C2680AB100207047F4
:10306000181D704703691960C2680132C260C269E5
:10307000134482690361934224BF436A03610021C0
:10308000FEF7D0BF38B504460D46E3683BB1626930
:10309000131D1268A3621344E362002038BD237A33
:1030A00033B929462046FEF7ADFF0028EDDA38BDDA
:1030B0006FF00100FBE70000C368C269013BC36019
:1030C0004369134482694361934224BF436A436165
:1030D00000238362036B03B11847704770B5202348
:1030E000044683F31188866A3EB9FFF7CBFF054695
:1030F00018B186F31188284670BDA36AE26A13F8F6
:10310000015BA362934202D32046FFF7D5FF002361
:1031100083F31188EFE700002DE9F84F04460E46CF
:1031200090469946202787F311880025AA46D4F8AF
:1031300028B0BBF1000F09D149462046FFF7A2FF96
:1031400020B18BF311882846BDE8F88FA16AE36AA5
:10315000A8EB050B5B1A9B4528BF9B46BBF1400FB4
:103160001BD9334601F1400251F8040B43F8040B1C
:103170009142F9D1A36A40334036A3624035A26A36
:10318000E36A9A4202D32046FFF796FF8AF311883A
:103190004545D8D287F31188C9E730465A46FDF72E
:1031A000F3FDA36A5B445E44A3625D44E7E700006D
:1031B00010B5029C0172043303FB0421C361002398
:1031C0008362C362039B0363049B00604060C4602E
:1031D00042610261816104624262436310BD00008A
:1031E000026AC260426A4261026100228262C26275
:1031F0006FF00101FEF722BF436902699A4203D1D1
:10320000C2680AB100207047184650F8043B0B60B2
:1032100070470000C368C2690133C3604369134447
:1032200082694361934224BF436A43610021FEF7F0
:10323000F9BE000038B504460D46E3683BB123698A
:103240001A1DA262E2691344E362002038BD237AAA
:1032500033B929462046FEF7D5FE0028EDDA38BD01
:103260006FF00100FBE7000003691960C268013AD2
:10327000C260C269134482690361934224BF436AF6
:10328000036100238362036B03B11847704700009A
:1032900070B5202304460E4683F31188856A35B93C
:1032A0001146FFF7C7FF10B185F3118870BDA36AFF
:1032B0001E70A36AE26A01339342A36204D3E169F8
:1032C00020460439FFF7D0FF002080F3118870BD3D
:1032D0002DE9F84F04460D4691469A464FF02008D6
:1032E00088F311880026B346A76A4FB95146204695
:1032F000FFF7A0FF20B187F311883046BDE8F88FB3
:10330000A06AE76AA9EB06033F1A9F4228BF1F463F
:10331000402F1BD905F1400355F8042B40F8042B2E
:103320009D42F9D1A36A4033A3624036A26AE36AA0
:103330009A4204D3E16920460439FFF795FF8BF3E5
:1033400011884E45D9D288F31188CDE729463A46EF
:10335000FDF71AFDA36A3B443D44A3623E44E5E702
:10336000026943699A4203D1C3681BB91846704782
:103370000023FBE7836A002BF8D0043B9B1AF5D0AF
:103380001360C368013BC360C3691A448369026167
:103390009A4224BF436A0361002383620123E5E765
:1033A00000F034B9034B002258631A610222DA603C
:1033B000704700BF000C0040014B0022DA607047EC
:1033C000000C0040014B5863704700BF000C0040E8
:1033D000FEE7000010B5174CFEF71AFDFEF73CFEA5
:1033E000802215492046FEF7C1FD012344F8180C40
:1033F0000374124B124AD96821F4E0610904090CE4
:103400000A431049DA60CA6842F08072CA600E4905
:103410000A6842F001020A601022DA77202283F85B
:103420002220002383F3118862B60848BDE81040CB
:10343000FEF7BEBDFC360020BC3C000800ED00E0FD
:103440000003FA05F0ED00E0001000E0C43C0008C5
:103450002DE9F84F1F4CDFF88090656904F11407DF
:103460004FF00008D9F82430266AAA689E1B9642BD
:103470001DD34FF0200AAA68236AD5F80CB0134474
:1034800023622B68BB425F60A6EB02066361C5F84E
:103490000C8001D1FFF790FF88F311882869D84785
:1034A0008AF311886569AB689E42E4D2DAE7626903
:1034B000BA420CD0916823628E1B9660A8680228DD
:1034C0002CBF1818981CBDE8F84FFFF77BBFBDE86C
:1034D000F88F00BFD4360020000C0040034B596821
:1034E0005A68521A9042FBD8704700BF001000E0A3
:1034F0004B6843608B688360CB68C3600B69436132
:103500004B6903628B6943620B680360704700007C
:1035100008B5224B22481A6940F2FF110A431A618A
:103520001A6922F4FF7222F001021A611A691A6BF9
:103530000A431A631A6D0A431A651A4A1B6D11462B
:10354000FFF7D6FF184802F11C01FFF7D1FF17481B
:1035500002F13801FFF7CCFF154802F15401FFF7E3
:10356000C7FF144802F17001FFF7C2FF124802F1D1
:103570008C01FFF7BDFF114802F1A801FFF7B8FF6A
:103580000F4802F1C401FFF7B3FF0E4802F1E0015A
:10359000FFF7AEFFBDE8084000F0A4B800380240D5
:1035A00000000240E43C0008000402400008024021
:1035B000000C0240001002400014024000180240BB
:1035C000001C02400020024008B500F0FFF9FFF7A0
:1035D00001FFFFF739F8BDE80840FEF7C5BE00005F
:1035E00070470000084B1A69920710B508D50024EF
:1035F0001C61202383F31188FFF72AFF84F31188CD
:10360000BDE81040FFF742B8000C0040104B1A6CA8
:1036100042F008021A641A6E42F008021A660D4A55
:103620001B6E936843F0080393600B4B53229A621E
:103630004FF0FF32DA6200229A615A63DA605A6010
:1036400001225A6108211A603220FDF7ABBD00BF8C
:1036500000380240002004E0000C00401F4B1A69B3
:103660006FEAC2526FEAD2521A611A69C2F30802B3
:103670001A614FF0FF301A695A69586100215A697E
:1036800059615A691A6A62F080521A621A6A02F023
:1036900080521A621A6A5A6A58625A6A59625A6A97
:1036A0001A6C42F080521A641A6E42F080521A6606
:1036B0001A6E0B4A106840F480701060186F00F4A6
:1036C0004070B0F5007F1EBF4FF480301867196757
:1036D000536823F40073536000F058B90038024077
:1036E00000700040324B4FF080521A64314A4FF460
:1036F000404111601A6842F001021A601A6892078C
:10370000FCD59A6822F003029A60294B19469A6800
:1037100012F00C02FBD1186800F0F90018609A60F2
:103720001A6842F480321A600B689B03FCD54B6F19
:1037300043F001034B671E4B5A6F9007FCD51E4A9E
:103740005A601A6842F080721A601A4A5368590423
:10375000FCD5174B1A689201FCD5184A9A600322CF
:10376000C3F88C20164B1A68164B9A42164B1BD185
:10377000164A1168164A914216D140F205121A6093
:103780000B4B9A6842F002029A609A6802F00C02AF
:10379000082AFAD15A6C42F480425A645A6E42F4B2
:1037A00080425A665B6E704740F20572E7E700BFE1
:1037B00000380240007000401854400700948838D8
:1037C000002004E011640020003C024000ED00E015
:1037D00041C20F41084A08B5536911680B4003F014
:1037E0000103536123B1054A13680BB15068984730
:1037F000BDE80840FEF74ABF003C014010410020F0
:10380000084A08B5536911680B4003F0020353617D
:1038100023B1054A93680BB1D0689847BDE80840CA
:10382000FEF734BF003C014010410020084A08B5B3
:10383000536911680B4003F00403536123B1054A37
:1038400013690BB150699847BDE80840FEF71EBFE9
:10385000003C014010410020084A08B55369116836
:103860000B4003F00803536123B1054A93690BB180
:10387000D0699847BDE80840FEF708BF003C01400A
:1038800010410020084A08B5536911680B4003F045
:103890001003536123B1054A136A0BB1506A98476C
:1038A000BDE80840FEF7F2BE003C01401041002098
:1038B000174B10B55C691A68144004F478725A61A9
:1038C000A30604D5134A936A0BB1D06A98476006E1
:1038D00004D5104A136B0BB1506B9847210604D5E1
:1038E0000C4A936B0BB1D06B9847E20504D5094A9B
:1038F000136C0BB1506C9847A30504D5054A936C23
:103900000BB1D06C9847BDE81040FEF7BFBE00BFBA
:10391000003C0140104100201A4B10B55C691A6848
:10392000144004F47C425A61620504D5164A136DB2
:103930000BB1506D9847230504D5134A936D0BB115
:10394000D06D9847E00404D50F4A136E0BB1506E4A
:103950009847A10404D50C4A936E0BB1D06E9847DA
:10396000620404D5084A136F0BB1506F98472304C3
:1039700004D5054A936F0BB1D06F9847BDE810404E
:10398000FEF784BE003C014010410020062108B52E
:103990000846FDF707FC06210720FDF703FC06217A
:1039A0000820FDF7FFFB06210920FDF7FBFB0621A0
:1039B0000A20FDF7F7FB06211720FDF7F3FB062190
:1039C0002820BDE80840FDF7EDBB000008B5FFF773
:1039D00045FE00F00DF8FDF78BFDFDF777FFFDF7D5
:1039E0004BFEFFF7FDFDBDE80840FFF7D9BC000026
:1039F000002304491A465A50C8180833802B4260E5
:103A0000F9D1704710410020034611F8012B03F84B
:103A1000012B002AF9D17047121012131211000065
:103A200053544D3332463F3F3F00000001203300E6
:103A30000010410101105A01031059010710310112
:103A400000000000203A00083F00000013040000BE
:103A5000803A00083F000000190400008A3A00087C
:103A60003F00000021040000943A00083F000000DD
:103A7000143700209C290020042E00206C320020E6
:103A800053544D3332463430780053544D3332461C
:103A90003432780053544D3332463434365858005B
:103AA0000096000000000000000000000000000080
:103AB0000000000000000000B9140008A514000870
:103AC000E1140008CD140008D9140008C51400083A
:103AD000B11400089D140008ED1400080000000057
:103AE000F1150008DD150008191600080516000874
:103AF00011160008FD150008E9150008D515000885
:103B00007516000800000000010000000000000021
:103B100002000000000000001D18000885180008C1
:103B200040004000AC3B0020BC3B002002000000F5
:103B3000000000000300000000000000C918000899
:103B40000000000010000000CC3B0020000000003E
:103B50000100000000000000A03E00200101020062
:103B600025424F41524425002553455249414C2599
:103B70000043756265426C61636B2D736F6C6F00FF
:103B80003031323334353637383941424344454693
:103B9000000000004865782F50726F6669434E43FD
:103BA0000043756265426C61636B2D424C000000FE
:103BB000092300087521000889170008ED22000874
:103BC00043000000C83B000809024300020100C096
:103BD0003209040000010202010005240010010561
:103BE00024010001042402020524060001070582C5
:103BF000030800FF09040100020A00000007050194
:103C00000240000007058102400000001200000091
:103C1000143C00081201100102000040AE2D0110FA
:103C20000002010203010000040309040040000037
:103C300000400000004000000040000000000100C3
:103C4000000002000000020000000200000002006C
:103C5000000002000000020000000200004000001E
:103C60000040000000400000004000000000010093
:103C7000000002000000020000000200000002003C
:103C8000000002000000020000000200000000002E
:103C9000111A0008F11C00089D1D0008400040009A
:103CA000003F0020003F002001000000103F0020E6
:103CB0008000000040010000030000006D61696E9B
:103CC00000000000DC3C0008183F002010410020EC
:103CD00001000000D13300080000000069646C6539
:103CE000000000000000802A00020000AAAAAAAA80
:103CF00000000000FFFF00000000000000A00A001C
:103D00000000000000000000AAAAAAAA000000000B
:103D1000FFFF0000000000000000000000000000A5
:103D200000000000AAAAAAAA00000000FFFF0000ED
:103D3000000000000000000080298A01000000004F
:103D4000AAAAAAAA40154501FFFF0000007070074B
:103D5000777000000080020100000000AAAAAAAA51
:103D600000400100FFFF000000000080080000008C
:103D70000000000000000000AAAAAAAA000000009B
:103D8000FFFF000000000000000000000000000035
:103D900000000000AAAAAAAA00000000FFFF00007D
:103DA0000000000000000000000000000000000013
:103DB0000A000000000000000300000000000000F6
:103DC00000000000000000000000000000000000F3
:103DD00000000000000000000000000000000000E3
:103DE000FF0096000000000804000000283C0008C6
:103DF00000000000000000000000000000000000C3
:083E00000000000000000000BA
:00000001FF
